:020000040000fa
:080000002c06040000000000c2
:020000040000fa
:020000040002f8
:04afe000dfff00008f
:020000040000fa
:020000040002f8
:04afe400ffff00006b
:020000040000fa
:020000040002f8
:04afe80078ff0000ee
:020000040000fa
:020000040002f8
:04afec007dff0000e5
:020000040000fa
:020000040002f8
:04aff00078ff0000e6
:020000040000fa
:1000080000000000000000000000000000000000e8
:1000180024060000000000000000000000000000ae
:1000280000000000000000000000000000000000c8
:100038000000000000000000000000009a09000015
:10004800cc0900000000000000000000960a000033
:100058000000000000000000000000000000000098
:100068000000000000000000000000000000000088
:100078000000000000000000000000000000000078
:10008800000000000000000000000000fc09000063
:100098002c0a000000000000000000000000000022
:1000a8000000000000000000000000000000000048
:1000b8000000000000000000000000000000000038
:1000c8000000000000000000000000000000000028
:1000d8000000000000000000000000000000000018
:1000e8000000000000000000000000000000000008
:1000f80000000000000000000000000000000000f8
:1001080000000000000000000000000000000000e7
:1001180000000000000000000000000000000000d7
:1001280000000000ce0a00000000000000000000ef
:1001380000000000000000000000000000000000b7
:1001480000000000000000000000000000000000a7
:100158000000000000000000000000000000000097
:100168000000000000000000000000000000000087
:100178000000000000000000000000000000000077
:100188000000000000000000000000000000000067
:100198000000000000000000020b00002e0b000011
:1001a8005a0b0000000000000000000000000000e2
:1001b8000000000000000000000000000000000037
:1001c8000000000000000000000000000000000027
:1001d8000000000000000000000000000000000017
:1001e8000000000000000000000000000000000007
:1001f80000000000000000000000000000000000f7
:1002080000000000000000000000000000000000e6
:1002180000000000000000000000000000000000d6
:1002280000000000000000000000000000000000c6
:1002380000000000000000000000000000000000b6
:1002480000000000000000000000000000000000a6
:100258000000000000000000000000000000000096
:100268000000000000000000000000000000000086
:0c0278000000000000000000000000007a
:020000040000fa
:10040000803e2000030007008100e900fcff3a0065
:1004100000000600831f7800c20320000400bc0017
:1004200066015100e0815900f23fb1000380b10044
:1004300006003500ee03090000000000423fb10055
:100440000380b100fbff3d001200b000223fb0006e
:10045000020035000280090000000000cf01780092
:1004600000000600889fbe008a9fbe008c1f780097
:100470000004be00a80107000478a30026003a008b
:100480006120e1002500320009f8a30025003a00b0
:100490006420e10021003200f507b1000508a30047
:1004a0000200320000004000818048006044b80033
:1004b000031020000200200000004000818048005e
:1004c0000805440089854c000a0541008b854900d8
:1004d0000a0550008b855800030033000a00be0057
:1004e00002047400838474008301d1000281d3006c
:1004f000830f7100f0ff3a008904d1000884d30013
:100500006001490082017800c1adde00fb07b00048
:1005100096010700070037000960a0000800be0030
:100520000400370012022000b28e8800f0ff2f0076
:10053000f1ff27004f0678004f05be004f04be00b4
:100540000000060004002000030037001400200013
:100550000100370014002000889fbe008a9fbe0063
:10056000841f7800640107004f00780011003300f9
:10057000f0ff2f00838f6c0006003b000405650030
:100580000a00a7000800370009f0a60010002000ac
:1005900008003700820f5400838f5c00030039008d
:1005a0001000200001003e000000200009f0a7001c
:1005b0000000ea004f05be004f04be000000e0004e
:1005c0000000060003f0a200869fbe00889fbe00c8
:1005d0008a9fbe008c9fbe0047010700890133003f
:1005e0006450e1004f0032006420e100520032000c
:1005f00003826c0007003b000905d0000306d00011
:10060000820f54000c065d00020039000200320027
:1006100089017800030678008582550004003d00ba
:100620000003fd008103fd008502ea008b85420086
:10063000840f720002003b0060001000e080180090
:100640006011b8000005eb007a28e1000a003900cb
:1006500006007800c75ddd00f707b20087807500ef
:100660002d003700828171000a0178006105600069
:100670008180d1000080d3008502e900f9ff3b00b2
:10068000060440008784480002003b006004140018
:10069000e0841c000988a300070032008a817100f1
:1006a00082817100610164008904d1000884d30053
:1006b0008b05e800170037000978a30013003a0003
:1006c0000b00e000130034008b05e900080444002f
:1006d00089844c000a4474000978a3000d003a0094
:1006e0000b00e000070034008b05e900080444001b
:1006f00089844c0001003a000b0020000978a30017
:10070000f7ff32000001eb00020037008281710028
:100710000a017800150107000cf0a70001f0a00005
:10072000410137006420e10002003a00838f6c0031
:10073000420133000801be000200be003a0137004a
:10074000869fbe00889fbe008a9fbe008c9fbe0011
:10075000e90007002b01330003866c006450e100c0
:100760002e0032006420e100330032006150e100cd
:100770002f0032006120e1003100320085855500f4
:10078000eb07b00009002000080420000500370036
:100790000804440089844c000a0031000603430029
:1007a00087834b000001530081815b00f8ff330019
:1007b0000203be000800a0000804440089844c0025
:1007c000f6ff3900c639dd008301730001003200f5
:1007d000130020008904d1000884d3000998a300e5
:1007e000050032000800a7000300a0008904d10022
:1007f0000884d3008b05e8008904d1000884d30065
:100800000001eb000281d200d800070001f0a10036
:100810000cf0a70001f0a000030137006420e10004
:10082000060132000801be000200be00f7ff3700db
:100830006120e100010132006000b800f3ff3700e1
:100840000000200001f82700f0ff3700869fbe005f
:10085000889fbe008a9fbe008c9fbe00a600070036
:10086000e800330003866c006450e100240032008d
:100870006420e100270032006150e10022003200d4
:100880006120e100210032008b854200eb07b100be
:100890000134b800003ab8000804420089844a00d4
:1008a000013ab8000030b8008880400009014a00d1
:1008b000040033000000400081804800020149002c
:1008c0008b05e900c909dd008301700001003200d9
:1008d00013002000c814de004814dd004709de00c4
:1008e0001200b200c808de00088470009f000700f4
:1008f00001f0a1000cf0a70001f0a000ca00370031
:100900006120e100cd0032000801be000200be00ff
:10091000f7ff37006150e100fcff3a00c7003700e5
:10092000829fbe000001be007b0007000470a7008c
:1009300003f0a1006509b100180032000e00350077
:100940006828e10007003500f0ff2f00f1ff2700c5
:100950000300e00015003b00010028004f01be002d
:100960000000050000004000818048008502e90089
:10097000fcff3a0009003700f88f420003003c00fa
:100980008000eb004f01be00000005008100d10097
:100990000080d3008502e800fcff3a000300e0007d
:1009a00002003b0060001000e08018004f01be0014
:1009b00000000600829fbe000001be005600070036
:1009c0000470a70003f0a10003f8a30015003a008b
:1009d0006509b100110032000a0035006928e10004
:1009e00003003500010028004f01be000000050093
:1009f00000004000818048008502e900fcff3a00c9
:100a000006003700f88f4200060035008100d10053
:100a10000080d3008502e800fcff3a004f01be00d1
:100a2000000006008000eb004f01be000000050042
:100a30000000fb00cf80de00020037000080fb00da
:100a40008000eb00829fbe00889fbe008a9fbe0090
:100a5000010578000100e0000400350008003c00ba
:100a60000000e000200032000500370060001000a8
:100a7000e080180002003b0001f024001a0037005b
:100a80000004be006011b8006b0920000982cf008d
:100a9000020039000882cf000441b00069425200d0
:100aa0000e00320008003b00828171006101640089
:100ab0008904d1000884d3008b05e8000442e800d3
:100ac000f9ff3a00050037000804440089844c000f
:100ad0008b05e9000442e900fbff3a002300070010
:100ae0000af0a70001f0a0004f05be004f04be00b1
:100af0004f01be00000006000004be000600070013
:100b00000003be000405be000200be000200070094
:100b1000844f750000000600c70ade00f107b2002e
:100b2000f50fb20008003200e1cf420002003200af
:100b30000170a00024000500810f70000100320048
:100b40000408050044000500810f700002003a000f
:100b5000140005008502e9000000400081c0480043
:100b6000fcff3b000170a000240005008100200074
:100b7000618055000b003d000b00200061fe2f003e
:100b80000100e1001d0034008281710061016400f8
:100b90008904d1000884d3000000e800faff3a007d
:100ba000710020006100640003007000020060001a
:100bb0000900320061044400e0844c000988a5006b
:100bc000050032008b05e8006808e10002003a00e9
:100bd0008904d1000884d300f20f20000258e100fc
:100be00005003d00c75ddd00f907b2008980750092
:100bf00008007800000006000bf827008b00780042
:100c0000000005000200be006450e100050036004f
:100c10006420e100020036000968a30001003a00e8
:100c20000800be000160a0004f06be004f05be00d8
:100c30004f04be004f03be0000000600f0ff2f006f
:100c4000f1ff2700f8ff37000020ef000220ef003f
:100c5000c088a900004006000f0021009027210055
:100c600000018800000000000000eb000007780091
:100c70000c000900002f78000007eb005420ef0063
:100c80000e2eef001e2eef0040a7a900a1002000ad
:100c9000dbfd0700e0022000303a880044e7a900ad
:100ca00044c7a9004407a9004427a9004447a90054
:100cb0004467a9004487a900300020000600fc001a
:100cc0003174200082072000a309200082487800a8
:100cd0008348780080487800113a80006180700075
:100ce0000600fc002174200062042000730520002f
:100cf0008248780083487800804878004427ef00d5
:100d0000e0022000303a8800300020000d00fc0096
:100d10003174200082072000a30920008248780057
:100d2000834878008048780000002000217420006b
:100d30006204200073052000824878008348780010
:100d40008048780042a7ae00feff3700813e2000b9
:100d5000abfd070010c0b30086e6b70090c2b30039
:100d6000c4e6b7000002200000708800007825006b
:100d70008070880010aea90010cea9004008a9001c
:100d80004028a9004048a9000008a9002008a9009f
:100d90004188a90041a8a90041c8a9002068a9006c
:100da00011a1a9001061a9001021a90010a1a8009b
:100db0001081a8000621ef00008020006008880054
:100dc00000e8a9004388a80043a8a90043c8a800d8
:100dd00020e8a80011e1a90013a1a9001221a9008f
:100de00012a1a8001281a8004408a8004428a90064
:100df0004448a9000a21ef000ea1ef000108a90054
:100e00002108a80013e1a8004d88a9004da8a90059
:100e10004dc8a9000368a9002368a9001fe1a90023
:100e200021e1a80021a1a90020c1a90020a1a800ba
:100e30002081a8002021a9001821ef00302d2400d6
:100e4000e00888004e08a9004e28a9004e48a800d6
:100e50000388a9002388a8002002a9002022a90055
:100e60002042a90020a2a9002062a9002082a90096
:100e700020e2a9002102a9002122a9007007200078
:100e80004011880022a2a90022c2a90022e2a900e2
:100e900021e2a8002182a9004588a90045a8a80050
:100ea00045c8a8002168a8002828a8002bc8a900c8
:100eb0002be8a9002c08a9000bc8a9000be8a90081
:100ec0000c08a90001eca90001aca900016ca90063
:100ed000014ca800012ca900010ca90000eca900fc
:100ee000008ca90000aca90000cca900000ca9004e
:100ef000002ca900004ca900006ca900202cef00d8
:100f0000402cef00602cef0020eca800200ca80083
:100f100040eca800400ca80060eca800600ca80001
:100f2000f07f200020608800020ca900022ca9009c
:100f3000024ca9000040200030618800462cef00e0
:100f4000662cef00282cef00482cef00682cef00f7
:100f50000aacef0023eca80023cca80043eca800c7
:100f600043cca90063eca80063cca90023aca90082
:100f7000238ca900dabc2a001b32240030002c008c
:100f8000fa608800fb60880020618800dabc2a00d3
:100f90001b32240020002c00fa608800fb608800cf
:100fa00010618800dabc2a001b32240030002c00bb
:100fb000fa608800fb60880020628800dabc2a00a2
:100fc0001b32240000002800fa608800fb608800c3
:100fd00010628800dabc2a001b32240030002c008a
:100fe000fa608800fb60880020638800dabc2a0071
:100ff0001b32240000002800fa608800fb60880093
:1010000010638800a70037003f0037000020200051
:10101000006188000020200000628800002020007d
:1010200000638800020ca900022ca800024ca80052
:1010300004acef0028acef0048acef0068acef0068
:10104000262cef00462cef00662cef000aacef00d8
:1010500023eca80023cca90043eca80043cca900b2
:1010600063eca80063cca900dabc2a001b32240080
:1010700030002c00fa608800fb6088002061880046
:10108000dabc2a001b32240000002800fa60880025
:10109000fb60880010618800dabc2a001b32240043
:1010a00030002c00fa608800fb6088002062880015
:1010b000dabc2a001b32240000002800fa608800f5
:1010c000fb60880010628800dabc2a001b32240012
:1010d00030002c00fa608800fb60880020638800e4
:1010e000dabc2a001b32240000002800fa608800c5
:1010f000fb6088001063880011eea90011aea90002
:10110000116ea9006700370035003700001020007d
:10111000006188000010200000628800001020009c
:1011200000638800020ca900022ca800024ca80051
:101130000a2cef0004acef00282cef0050552500de
:1011400040628800a0aa2a0040638800dabc2a0016
:101150001b32240030002c00fa608800fb608800fd
:1011600020618800dabc2a001b32240000002c0019
:10117000fa608800fb60880010618800dabc2a00f1
:101180001b32240030002c00fa608800fb608800cd
:1011900020628800dabc2a001b32240000002c00e8
:1011a000fa608800fb60880010628800dabc2a00c0
:1011b0001b32240030002c00fa608800fb6088009d
:1011c00020638800dabc2a001b32240000002c00b7
:1011d000fa608800fb6088001063880031003700e7
:1011e000300037000010200000618800001020004f
:1011f00000628800020ca900022ca800024ca80082
:101200000a2cef0004acef00282cef0000002400b3
:1012100040628800dabc2a001b32240030002c0017
:10122000fa608800fb60880020618800dabc2a0030
:101230001b32240000002c00fa608800fb6088004c
:1012400010618800dabc2a001b32240030002c0018
:10125000fa608800fb60880020628800dabc2a00ff
:101260001b32240000002c00fa608800fb6088001c
:1012700010628800dabc2a001b32240030002c00e7
:10128000fa608800fb60880020638800dabc2a00ce
:101290001b32240000002c00fa608800fb608800ec
:1012a00010638800218ca900418ca900618ca900e1
:1012b000216ca900416ca900616ca900214ca90016
:1012c000414ca900614ca90020eca80040eca8000a
:1012d00060eca8003e2cef005e2cef007e2cef00af
:1012e00001eca8000000eb0041622100ff000900b2
:1012f000805878000572ef000672ef008003070047
:1013000010c0b300eef1b70010c0b300eff1b700aa
:101310007d070700e431ef00e031ef00e231ef003c
:10132000f209070010cea90014cea8009809070002
:10133000f6003700ff3ffc004200f8003600f800de
:101340004400f8008e1f78000e0020000d000900f8
:10135000be1f78003200f8000100fc0000e8a90080
:10136000f08e800060088800e031ec00ff3ffc0058
:101370003200f900ae0120000d0009004f1778007f
:101380004f0778004400f9003600f9004200f900e8
:101390000100fc0000400600ff3ffc004200f80096
:1013a0003600f8004400f8008e1f78000e00200080
:1013b0000d000900be1f78003200f8000100fc009b
:1013c0000108a900128eaa00108ea900ff3ffc00a0
:1013d0003200f900ae0120000d0009004f1778001f
:1013e0004f0778004400f9003600f9004200f90088
:1013f0000100fc0000400600ff3ffc004200f80036
:101400003600f8004400f8008e1f78000e0020001f
:101410000d000900be1f78003200f8000100fc003a
:101420000368a9002368a9001fe1a900ff3ffc0091
:101430003200f900ae0120000d0009004f177800be
:101440004f0778004400f9003600f9004200f90027
:101450000100fc0000400600ff3ffc004200f800d5
:101460003600f8004400f8008e1f78000e002000bf
:101470000d000900be1f78003200f8000100fc00da
:101480000388a9002132ae00110037002072ec0061
:101490002012ae00070037001fd2bf000080fb0003
:1014a00000004000413221006080780030638800f5
:1014b000060037001ed2bf000080fb000000400085
:1014c00041322100608078003063880006003700d8
:1014d0002072ef00628f8000020141004032210043
:1014e00060007900306388001dd2bf000080fb00df
:1014f000000040004122210060807800e008880060
:10150000ff3ffc003200f900ae0120000d00090091
:101510004f1778004f0778004400f9003600f900b3
:101520004200f9000100fc0000400600ff3ffc0003
:101530004200f8003600f8004400f8008e1f7800e2
:101540000e0020000d000900be1f78003200f800d8
:101550000100fc000168a9000572ec0005d2bf0083
:101560008080fb0030118000426221008070790091
:10157000ff3ffc003200f900ae0120000d00090021
:101580004f1778004f0778004400f9003600f90043
:101590004200f9000100fc0000400600ff3ffc0093
:1015a0004200f8003600f8004400f8008e1f780072
:1015b0000e0020000d000900be1f78003200f80068
:1015c0000100fc000828a9002242ae0000003700fc
:1015d0002222af002222a900ff3ffc003200f900c6
:1015e000ae0120000d0009004f1778004f0778006a
:1015f0004400f9003600f9004200f9000100fc0047
:1016000000400600ff3ffc004200f8003600f800f2
:101610004400f8008e1f78000e0020000d00090025
:10162000be1f78003200f8000100fc000bc8a900c2
:10163000ff3ffc003200f900ae0120000d00090060
:101640004f1778004f0778004400f9003600f90082
:101650004200f9000100fc0000400600ff3ffc00d2
:101660004200f8003600f8004400f8008e1f7800b1
:101670000e0020000d000900be1f78003200f800a7
:101680000100fc000be8a900ff3ffc003200f9005c
:10169000ae0120000d0009004f1778004f077800b9
:1016a0004400f9003600f9004200f9000100fc0096
:1016b00000400600ff3ffc004200f8003600f80042
:1016c0004400f8008e1f78000e0020000d00090075
:1016d000be1f78003200f8000100fc000c08a900d1
:1016e000ff3ffc003200f900ae0120000d000900b0
:1016f0004f1778004f0778004400f9003600f900d2
:101700004200f9000100fc00004006007f080700cd
:1017100023d2bf0007f2b70070cbb3000752b50069
:1017200006003900e0cfb3000752b50001003900d0
:10173000010037000872ef00d800370007f2ae0052
:10174000370037000872ef0060c8b3000752e300ab
:1017500005003a0007d2bf0008f2b70009f2ef0017
:101760000af2ef002d00370060c9b3000752e30012
:1017700005003a0007d2bf0008f2b7000bf2ef00f5
:101780000cf2ef002500370060cab3000752e300f7
:1017900005003a0007d2bf0008f2b7000df2ef00d3
:1017a0000ef2ef001d00370060cbb3000752e300dc
:1017b00005003a0007d2bf0008f2b7000ff2ef00b1
:1017c00010f2ef001500370060ccb3000752e300c1
:1017d00004003a0007d2bf0008f2b70011f2ef0090
:1017e0000e00370060cdb3000752e30004003a005a
:1017f00007d2bf0008f2b70012f2ef00070037006f
:1018000060ceb3000752e30004003a0007d2bf00e5
:1018100008f2b70013f2ef0014f2ef009f00370058
:101820000852e20002003a009c0037009b0037009b
:1018300060c8b3000852e3003a003a0000e0ef004d
:101840000952e30003003a0007d2bf0009f2b700d3
:10185000330037000752ec000af2b70009d2bf008c
:101860001752b5002d003a00e411e2000a003600dc
:101870000ad2bf0071fc07000001be00a08f8000eb
:10188000b18f8000aefb07000090880011908800a7
:10189000e431ef000c0037000ad2bf0067fc0700fc
:1018a0000001be00508f800065fc0700a4fb07000c
:1018b0000090880011908800508f800060fc070025
:1018c000a08f8800b18f8800a08f8000b18f80002a
:1018d00038fc070016f2b70016d2bf000080fb00ec
:1018e00000004000413221006080780030628800b2
:1018f0002132a90003f2af0005003700e451a8002f
:10190000e031ef00e231ef0011e1a8000300370001
:1019100014cea90011e1a9001772ef0009f2ef003f
:101920005e00370060c9b3000852e30042003a008d
:1019300000e0ef000b52e30003003a0007d2bf00c3
:101940000bf2b7003b00370007d2bf000cf2b70024
:101950000bd2bf0041c3b30080cf1000340036006b
:10196000a0c6b3000b52e30031003e000bd2bf0013
:1019700017f2b7000cd2bf000080fb00408f880038
:101980001ad2bf000080fb00c200dd0040422100ef
:10199000008040001000be000001be000cd2bf005d
:1019a00023fc0700a9fb0700ddfb0700508f880020
:1019b000e431ef002212af0010003700f431ef00e5
:1019c000f631ef00462cef00e411a80019d2bf0059
:1019d0001afc07000001be00408f800018fc0700c1
:1019e00057fb0700c08f8800d18f8800e031ef00df
:1019f000e231ef0011e1a8000c003700528f8000a7
:101a0000020141004032210060007900306288000c
:101a1000508f80000afc0700a08f8800b18f8800db
:101a2000e031ef00e231ef0011e1a90014cea8008f
:101a30000bf2ef001900370060cab3000852e30050
:101a40000a003a0000e0ef000d52e30003003a0004
:101a500007d2bf000df2b7000300370007d2bf0066
:101a60000ef2b700c60007000c00370060cbb300d1
:101a70000852e30009003a0000e0ef000f52e300d3
:101a800003003a0007d2bf000ff2b700030037008f
:101a900007d2bf0010f2b700bf000700118f80000f
:101aa000008f8000808f50009f003100e231ec00f9
:101ab000218f8000e18f500048003a00408f800065
:101ac000dffb07000001be00a08f8000b18f800007
:101ad0009efa070040003c00a28f8000b38f800078
:101ae000c08f8000d18f8000b7fa0700a08f8800d8
:101af000b18f8800a28f8000b38f8000408f80005c
:101b0000cffb070091fa070029003c00408f8000be
:101b1000cbfb0700a08f8800b18f8800428f800028
:101b200002014100403221006000790030628800eb
:101b3000508f8000e811b500c1fb0700808f88003e
:101b4000918f88001bd2bf00bcfb07000001be00c4
:101b5000808f8000918f8000f9fa0700e08f880065
:101b6000f18f8800e031ef00e231ef00e431ef0067
:101b70006011b800e08f8000f18f800071fa0700db
:101b800007003a00528f80000201410040322100dc
:101b9000600079003062880011e1a900020037007e
:101ba000e431a80011e1a8002132a8000a003700a2
:101bb000a08f8000b18f80007efb070016f2b70077
:101bc00016d2bf000080fb0000004000413221001f
:101bd000608078003062880053003700218f8000d9
:101be000e28f50002b003a00a08f8000b18f800060
:101bf000e28f8000f38f800072fa0700a08f8800c8
:101c0000b18f8800f7f1ae0002003700f431ef0029
:101c1000f631ef00a28f8000b38f8000508f8000dc
:101c200087fb07004bfa07000c003d00a08f8000e7
:101c3000b18f80005ffb070016f2b70016d2bf001d
:101c40000080fb00000040004132210060807800ed
:101c50003062880011e1a8000d003700528f80002b
:101c600002014100403221006000790030628800aa
:101c7000e431ef00e031ef00e231ef0011e1a900c3
:101c8000508f80006efb0700a08f8800b18f880006
:101c900025003700218f8000e48f500022003a0099
:101ca000a08f8000b18f8000029080001390800090
:101cb00044fa0700a08f8800b18f8800020020003e
:101cc00003002000a08f8000b18f80001ffa070062
:101cd0000a003c0014cea900e431ef00462cef00ce
:101ce0001772ef00e031ef00e231ef00f431ef0066
:101cf000f631ef0011e1a9000b003700a08f800042
:101d0000b18f80002bfb070016f2b70016d2bf0080
:101d10000080fb000000400041322100608078001c
:101d20003062880011e1a800e411af00040ea800a1
:101d3000e411ae00040ea900e431af00042ea800a7
:101d4000e431ae00042ea900e451af00142ea80027
:101d5000e451ae00142ea900e411e20006003a009e
:101d60001752e20002003600140ea80001003700ee
:101d7000140ea90001003700140ea90063fe3700fd
:101d80000df2ef000000060011f2ef000000060067
:101d900012f2ef0000000600b0c7b3000f52e300dc
:101da00002003a00e5060700d30037000fd2bf005b
:101db00080407800e5cf500026003a0010d2bf00e6
:101dc0001cf2b7001c72d5001c52e20008003a0059
:101dd0000388a9002388a900628f800002014100c6
:101de000403221006000790030638800180037001d
:101df000618f80001cd2bf000080fb00810f50006b
:101e0000020036001e72ef00030037001cd2bf0034
:101e1000ec51b5001ef2b700618f80001cd2bf00ec
:101e20000080fb000100400080007800f0072000e7
:101e3000808f500003003600f0c7b3001ff2b700d8
:101e400003003700608f80001c52b4001ff2b700ff
:101e5000a90037000fd2bf0080407800e6cf5000c5
:101e600016003a0010d2bf001df2b7001052e20077
:101e70000a0036001821ef000388a9001dd2bf0018
:101e80000080fb00000040004122210060807800bb
:101e9000e00888002388a800070037000388a9000d
:101ea0002388a900628f8000020141004032210096
:101eb00060007900306388008f0037000fd2bf00c8
:101ec00080407800e7cf500022003a0010d2bf00d7
:101ed0000080fb00608f8800618f80001cd2bf00f3
:101ee0000080fb00810f5000020036001e72ef00e0
:101ef000030037001cd2bf00ec51b5001ef2b70042
:101f0000618f80001cd2bf000080fb0001004000f8
:101f100080007800f0072000808f5000030036001a
:101f2000f0c7b3001ff2b70003003700608f8000d6
:101f30001c52b4001ff2b70010d2bf000080fb009b
:101f4000000040004132210060807800306388004a
:101f5000690037000fd2bf0080407800ebcf5000ff
:101f600007003a001012af00020037002212a90049
:101f7000020037002212a800e431ef005e003700b3
:101f80000fd2bf0080407800efcf500008003a0029
:101f900010d2bf0018f2b70018d2bf000080fb00bb
:101fa0000020ec004400dd00f08e88005200370075
:101fb0000fd2bf0080407800f0cf500003003a00fd
:101fc0001052ec0019f2b7004b0037000fd2bf00df
:101fd00080407800f1cf500008003a001052ec0029
:101fe0001af2b70000c8b3001a52b5000200390057
:101ff000f0c7b3001af2b7003f0037000fd2bf009e
:1020000080407800f2cf500003003a001052ec00fc
:102010001bf2b7003800370020c4b3000f52e300b2
:1020200007003a001052e20002003a004d06070095
:1020300002003700048ea8007d0607002e0037003e
:1020400000c5b3000f52e3002b003a0014cea800e5
:102050001052ec00eef1b700eed1bf000080fb00a3
:102060004500de00eef1b700efd1bf00ee51e30016
:102070002100320014cea900462cef001772ef00a9
:10208000ee51e20002003a001f050700170037007a
:10209000eed1bf0080407800e1cf500002003a004e
:1020a0001904070011003700eed1bf00804078000e
:1020b000e2cf500002003a00130307000b00370084
:1020c000eed1bf0080407800e3cf500002003a001c
:1020d0000d02070005003700eed1bf0080407800f8
:1020e000e4cf500001003a0007010700eed1bf0025
:1020f000eff1b70014cea8000ff2ef0000000600c9
:1021000000d0270020918800a0c7250030918800ca
:10211000509825004091880040812500509188000a
:10212000906a2500609188003054250070918800e5
:10213000303e2500809188009028250090918800ed
:1021400050132500a091880060fe2400b091880003
:10215000c0e92400c091880080d52400d091880077
:1021600090c12400e0918800f0ad2400f091880037
:10217000a09a240000928800a08724001092880072
:10218000f07424002092880090622400309288002d
:102190008050240040928800b03e24005092880075
:1021a000302d240060928800f01b2400709288007b
:1021b000000b24008092880050fa2300909288003f
:1021c000e0e92300a0928800c0d92300b0928800e3
:1021d000e0c92300c092880040ba2300d092880052
:1021e000e0aa2300e0928800c09b2300f0928800c0
:1021f000e08c230000938800307e23001093880039
:10220000d06f230020938800a061230030938800c2
:10221000b053230040938800f0452300509388007a
:102220007038230060938800202b2300709388006f
:10223000101e230080938800401123009093880093
:1022400090042300a093880020f82200b093880017
:10225000e0eb2200c0938800d0df2200d0938800fa
:10226000f0d32200e093880050c82200f093880049
:10227000d0bc22000094880080b122001094880015
:1022800070a6220020948800809b22003094880051
:10229000c09022004094880020862200509488003c
:1022a000c07b2200609488008071220070948800b6
:1022b0006067220080948800805d220090948800ee
:1022c000c0532200a0948800204a2200b0948800c5
:1022d000b0402200c094880060372200d09488006b
:1022e000402e2200e094880040252200f0948800cf
:1022f000601c220000958800b01322001095880011
:10230000200b220020958800b00222003095880022
:1023100060fa21004095880040f221005095880025
:1023200030ea21006095880050e221007095880015
:1023300090da210080958800e0d2210090958800f5
:1023400060cb2100a0958800f0c32100b0958800e3
:10235000b0bc2100c095880080b52100d0958800d0
:1023600080ae2100e095880090a72100f0958800bc
:10237000b0a0210000968800009a210010968800e5
:102380006093210020968800e08c21003096880020
:102390008086210040968800308021005096880079
:1023a000007a210060968800f07321007096880002
:1023b000f06d2100809688000068210090968800ca
:1023c00040622100a0968800805c2100b0968800c1
:1023d000e0562100c096880060512100d096880008
:1023e000f04b2100e096880090462100f09688008e
:1023f0005041210000978800203c21001097880060
:102400001037210020978800103221003097880073
:10241000202d2100409788004028210050978800f7
:102420008023210060978800d01e210070978800cb
:10243000301a210080978800a0152100909788000d
:1024400020112100a0978800c00c2100b0978800bf
:1024500070082100c097880020042100d0978800d0
:10246000f0ff2000e0978800d0fb2000f097880064
:10247000c0f7200000988800d0f320001098880052
:10248000e0ef20002098880000ec200030988800c1
:1024900030e820004098880070e4200050988800c0
:1024a000c0e020006098880020dd2000709888003f
:1024b00090d920008098880010d62000909888003d
:1024c000a0d22000a098880040cf2000b0988800bb
:1024d000e0cb2000c0988800a0c82000d0988800d9
:1024e00060c52000e098880030c22000f098880085
:1024f00010bf20000099880000bc200010998800bf
:1025000000000600000006002433ef001000200049
:102510003099880020002000409988003000200079
:102520005099880030002000609988003000200019
:1025300070998800300020008099880030002000c9
:102540009099880030002000a09988004000200069
:10255000b099880040002000c09988004000200009
:10256000d099880040002000e099880040002000b9
:10257000f099880050002000009a88005000200048
:10258000109a880050002000209a880050002000f7
:10259000309a880060002000409a88006000200087
:1025a000509a880060002000609a88007000200027
:1025b000709a880070002000809a880070002000c7
:1025c000909a880080002000a09a88008000200057
:1025d000b09a880090002000c09a880090002000e7
:1025e000d09a8800a0002000e09a8800a000200077
:1025f000f09a8800b0002000009b8800c0002000f6
:10260000109b8800c0002000209b8800d000200084
:10261000309b8800e0002000409b8800e000200004
:10262000509b8800f0002000609b88000001200083
:10263000709b880010012000809b880020012000f2
:10264000909b880030012000a09b88004001200062
:10265000b09b880050012000c09b880060012000d2
:10266000d09b880070012000e09b88009001200032
:10267000f09b8800a0012000009c8800b001200091
:10268000109c8800d0012000209c8800e0012000e0
:10269000309c880000022000409c8800200220001e
:1026a000509c880040022000609c8800600220004e
:1026b000709c880080022000809c8800a00220007e
:1026c000909c8800c0022000a09c8800f00220009e
:1026d000b09c880010032000c09c880040032000ac
:1026e000d09c880070032000e09c8800a00320009c
:1026f000f09c8800d0032000009d8800100420007a
:10270000109d880040042000209d88008004200047
:10271000309d8800c0042000409d880000052000f6
:10272000509d880050052000609d8800a005200075
:10273000709d8800e0052000809d880040062000f4
:10274000909d880090062000a09d8800f006200043
:10275000b09d880050072000c09d8800c007200061
:10276000d09d880030082000e09d8800a00820004f
:10277000f09d880020092000009e8800a00920000c
:10278000109e8800200a2000209e8800b00a2000a9
:10279000309e8800500b2000409e8800f00b2000e7
:1027a000509e8800900c2000609e8800400d200004
:1027b000709e8800000e2000809e8800c00e2000c1
:1027c000909e8800a00f2000a09e8800701020001e
:1027d000b09e880060112000c09e8800501220002a
:1027e000d09e880060132000e09e880070142000b6
:1027f000f09e880090152000009f8800c0162000e1
:10280000109f880000182000209f88006019200079
:10281000309f8800c01a2000409f8800401c200084
:10282000509f8800d01d2000609f8800701f2000ee
:10283000709f880030212000809f88001023200096
:10284000909f880000252000a09f8800102720006e
:10285000b09f880030292000c09f8800802b200076
:10286000d09f8800f02d2000e09f8800703020006d
:10287000f09f88002033200000a088000036200050
:1028800010a088000039200020a08800203c2000f3
:1028900030a08800703f200040a088000043200046
:1028a00050a08800b046200060a08800a04a200008
:1028b00070a08800c04e200080a088002053200017
:1028c00090a08800c0572000a0a08800a05c200035
:1028d000b0a08800c0612000c0a088002067200050
:1028e000d0a08800e06c2000e0a08800e07220000a
:1028f000f0a088004079200000a18800f07f20002f
:1029000010a18800000006002433ef0060002000c2
:1029100030998800700020004099880080002000d5
:102920005099880080002000609988008000200075
:102930007099880090002000809988009000200005
:1029400090998800a0002000a0998800a000200095
:10295000b0998800b0002000c0998800b000200025
:10296000d0998800c0002000e0998800c0002000b5
:10297000f0998800d0002000009a8800d000200044
:10298000109a8800e0002000209a8800f0002000c3
:10299000309a8800f0002000409a88000001200052
:1029a000509a880010012000609a880010012000d1
:1029b000709a880020012000809a88003001200051
:1029c000909a880040012000a09a880050012000c1
:1029d000b09a880060012000c09a88007001200031
:1029e000d09a880080012000e09a880090012000a1
:1029f000f09a8800a0012000009b8800b001200010
:102a0000109b8800d0012000209b8800e00120005e
:102a1000309b8800f0012000409b880010022000bd
:102a2000509b880020022000609b8800400220000c
:102a3000709b880050022000809b8800700220005c
:102a4000909b880090022000a09b8800b00220008c
:102a5000b09b8800d0022000c09b8800f0022000bc
:102a6000d09b880010032000e09b880030032000ea
:102a7000f09b880060032000009c880080032000f9
:102a8000109c8800b0032000209c8800d003200008
:102a9000309c880000042000409c88003004200006
:102aa000509c880060042000609c880090042000f6
:102ab000709c8800d0042000809c880000052000c5
:102ac000909c880040052000a09c88008005200084
:102ad000b09c8800c0052000c09c88000006200033
:102ae000d09c880050062000e09c880090062000c2
:102af000f09c8800e0062000009d88003007200040
:102b0000109d880080072000209d8800e00720009d
:102b1000309d880040082000409d8800a0082000cb
:102b2000509d880000092000609d880070092000e9
:102b3000709d8800e0092000809d8800500a2000d8
:102b4000909d8800d00a2000a09d8800500b200096
:102b5000b09d8800d00b2000c09d8800600c200034
:102b6000d09d8800f00c2000e09d8800800d2000a2
:102b7000f09d8800200e2000009e8800c00e2000de
:102b8000109e8800700f2000209e880030102000ca
:102b9000309e8800f0102000409e8800b011200078
:102ba000509e880080122000609e880060132000e4
:102bb000709e880040142000809e88003015200000
:102bc000909e880020162000a09e880030172000cc
:102bd000b09e880040182000c09e88006019200028
:102be000d09e8800801a2000e09e8800c01b200034
:102bf000f09e8800001d2000009f8800601e2000bd
:102c0000109f8800c01f2000209f880030212000d6
:102c1000309f8800c0222000409f88005024200060
:102c2000509f880000262000609f8800c027200059
:102c3000709f880090292000809f8800802b2000b2
:102c4000909f8800802d2000a09f8800902f20005a
:102c5000b09f8800c0312000c09f88001034200041
:102c6000d09f880070362000e09f88000039200047
:102c7000f09f8800903b200000a08800503e20007c
:102c800010a088003041200020a08800304420009f
:102c900030a088005047200040a08800a04a2000b3
:102ca00050a08800104e200060a08800a051200095
:102cb00070a088006055200080a088005059200036
:102cc00090a08800705d2000a0a08800c061200056
:102cd000b0a0880040662000c0a08800f06a2000f4
:102ce000d0a08800e06f2000e0a0880000752000e0
:102cf000f0a08800607a200000a18800f07f20000a
:102d000010a18800000006002433ef0050012000cd
:102d100030998800700120004099880080012000cf
:102d2000509988009001200060998800900120004f
:102d300070998800a001200080998800b0012000cf
:102d400090998800c0012000a0998800d00120003f
:102d5000b0998800e0012000c0998800000220009e
:102d6000d099880010022000e099880020022000fd
:102d7000f099880030022000009a8800400220006c
:102d8000109a880060022000209a880070022000bb
:102d9000309a880090022000409a8800a00220000b
:102da000509a8800c0022000609a8800d00220005b
:102db000709a8800f0022000809a8800100320009a
:102dc000909a880020032000a09a880040032000e9
:102dd000b09a880060032000c09a88008003200019
:102de000d09a8800a0032000e09a8800c003200049
:102df000f09a8800e0032000009b88001004200067
:102e0000109b880030042000209b88006004200074
:102e1000309b880080042000409b8800b004200084
:102e2000509b8800e0042000609b88000005200083
:102e3000709b880030052000809b88006005200082
:102e4000909b8800a0052000a09b8800d005200052
:102e5000b09b880000062000c09b88004006200030
:102e6000d09b880070062000e09b8800b006200000
:102e7000f09b8800f0062000009c880030072000ae
:102e8000109c880070072000209c8800c00720004c
:102e9000309c880000082000409c880050082000da
:102ea000509c8800a0082000609c8800f00820004a
:102eb000709c880040092000809c8800a0092000a8
:102ec000909c8800f0092000a09c8800500a2000f7
:102ed000b09c8800b00a2000c09c8800100b200025
:102ee000d09c8800800b2000e09c8800f00b200024
:102ef000f09c8800600c2000009d8800d00c200011
:102f0000109d8800400d2000209d8800c00d2000ed
:102f1000309d8800400e2000409d8800c00e20009b
:102f2000509d8800500f2000609d8800e00f200019
:102f3000709d880070102000809d88001011200076
:102f4000909d8800b0112000a09d880050122000a4
:102f5000b09d880000132000c09d8800b0132000a1
:102f6000d09d880070142000e09d8800301520005e
:102f7000f09d8800f0152000009e8800c0162000fb
:102f8000109e8800a0172000209e88007018200046
:102f9000309e880060192000409e8800501a200052
:102fa000509e8800401b2000609e8800401c20002e
:102fb000709e8800401d2000809e8800601e2000ba
:102fc000909e8800701f2000a09e8800a0202000f6
:102fd000b09e8800d0212000c09e880010232000d1
:102fe000d09e880050242000e09e8800b02520005c
:102ff000f09e880010272000009f88008028200075
:10300000109f8800f0292000209f8800802b20003e
:10301000309f8800102d2000409f8800c02e200087
:10302000509f880070302000609f88004032200050
:10303000709f880010342000809f88000036200098
:10304000909f8800f0372000a09f8800003a200061
:10305000b09f8800203c2000c09f8800503e200088
:10306000d09f8800a0402000e09f880000432000ff
:10307000f09f88007045200000a0880000482000d4
:1030800010a08800a04a200020a08800604d2000e9
:1030900030a088003050200040a08800205320003d
:1030a00050a088003056200060a0880050592000b1
:1030b00070a08800a05c200080a088000060200034
:1030c00090a0880080632000a0a0880020672000d6
:1030d000b0a08800f06a2000c0a08800d06e200058
:1030e000d0a08800e0722000e0a0880020772000b7
:1030f000f0a08800807b200000a18800f07f2000e5
:1031000010a18800000006002433ef0040042000d6
:1031100030998800600420004099880080042000d5
:1031200050998800a004200060998800c004200005
:1031300070998800e0042000809988000005200034
:103140009099880030052000a09988005005200043
:10315000b099880070052000c0998800a005200063
:10316000d0998800c0052000e0998800e005200083
:10317000f099880010062000009a88004006200080
:10318000109a880060062000209a8800900620008f
:10319000309a8800c0062000409a8800f00620007f
:1031a000509a880020072000609a8800500720006d
:1031b000709a880080072000809a8800c00720004d
:1031c000909a8800f0072000a09a8800300820001c
:1031d000b09a880060082000c09a8800a0082000eb
:1031e000d09a8800e0082000e09a8800200920009a
:1031f000f09a880050092000009b8800a009200058
:10320000109b8800e0092000209b8800200a2000f5
:10321000309b8800700a2000409b8800b00a200084
:10322000509b8800000b2000609b8800500b200002
:10323000709b8800a00b2000809b8800f00b200072
:10324000909b8800400c2000a09b8800900c2000e0
:10325000b09b8800f00c2000c09b8800400d20002f
:10326000d09b8800a00d2000e09b8800000e20006d
:10327000f09b8800600e2000009c8800c00e20009b
:10328000109c8800300f2000209c8800a00f200098
:10329000309c880000102000409c880070102000a6
:1032a000509c8800f0102000609c88006011200075
:1032b000709c8800e0112000809c88005012200043
:1032c000909c8800e0122000a09c880060132000e1
:1032d000b09c8800e0132000c09c8800701420007f
:1032e000d09c880000152000e09c880090152000ec
:1032f000f09c880020162000009d8800c016200049
:10330000109d880060172000209d88000018200074
:10331000309d8800b0182000409d88006019200072
:10332000509d8800101a2000609d8800c01a20005f
:10333000709d8800801b2000809d8800401c20001c
:10334000909d8800001d2000a09d8800d01d2000b9
:10335000b09d8800a01e2000c09d8800701f200026
:10336000d09d880050202000e09d88003021200062
:10337000f09d880020222000009e8800102320005d
:10338000109e880000242000209e88000025200038
:10339000309e880000262000409e880010272000d4
:1033a000509e880020282000609e88003029200040
:1033b000709e8800502a2000809e8800802b20006c
:1033c000909e8800b02c2000a09e8800f02d200048
:1033d000b09e8800302f2000c09e880070302000f2
:1033e000d09e8800c0312000e09e8800203320005d
:1033f000f09e880090342000009f88000036200056
:10340000109f880070372000209f8800003920001e
:10341000309f8800803a2000409f8800203c200098
:10342000509f8800c03d2000609f8800703f2000b2
:10343000709f880030412000809f8800004320005a
:10344000909f8800d0442000a09f8800b0462000b4
:10345000b09f8800a0482000c09f8800a04a20009c
:10346000d09f8800b04c2000e09f8800c04e200014
:10347000f09f8800f050200000a08800205320001a
:1034800010a088006055200020a08800c0572000b0
:1034900030a08800205a200040a08800a05c2000b6
:1034a00050a08800205f200060a08800c06120003c
:1034b00070a088006064200080a088002067200041
:1034c00090a08800006a2000a0a08800e06c200086
:1034d000b0a08800e06f2000c0a08800e07220004b
:1034e000d0a0880010762000e0a08800407920005d
:1034f000f0a08800907c200000a18800f07f2000d0
:1035000010a18800000006002433ef0040062000d0
:1035100030998800800d200040998800c00d20005f
:1035200050998800000e200060998800400e20000d
:1035300070998800800e200080998800c00e2000bd
:1035400090998800100f2000a0998800500f20004b
:10355000b0998800a00f2000c0998800e00f2000db
:10356000d099880030102000e09988007010200069
:10357000f0998800c0102000009a880010112000e7
:10358000109a880060112000209a8800b011200055
:10359000309a880000122000409a880050122000c3
:1035a000509a8800b0122000609a88000013200012
:1035b000709a880060132000809a8800b013200061
:1035c000909a880010142000a09a8800701420009f
:1035d000b09a8800d0142000c09a880030152000ce
:1035e000d09a880090152000e09a8800f0152000fd
:1035f000f09a880060162000009b8800c01620000a
:10360000109b880030172000209b8800a017200006
:10361000309b880000182000409b88007018200014
:10362000509b8800e0182000609b880060192000f3
:10363000709b8800d0192000809b8800501a2000c1
:10364000909b8800c01a2000a09b8800401b20008f
:10365000b09b8800c01b2000c09b8800401c20003d
:10366000d09b8800c01c2000e09b8800401d2000eb
:10367000f09b8800d01d2000009c8800601e200068
:10368000109c8800e01e2000209c8800701f2000f5
:10369000309c880010202000409c8800a020200042
:1036a000509c880030212000609c8800d0212000a0
:1036b000709c880070222000809c880010232000cd
:1036c000909c8800b0232000a09c880050242000fb
:1036d000b09c880000252000c09c8800b0252000f8
:1036e000d09c880060262000e09c880010272000e5
:1036f000f09c8800c0272000009d880080282000c2
:10370000109d880030292000209d8800f02920008d
:10371000309d8800c02a2000409d8800802b20001a
:10372000509d8800502c2000609d8800102d2000a6
:10373000709d8800f02d2000809d8800c02e200004
:10374000909d8800902f2000a09d88007030200060
:10375000b09d880050312000c09d8800403220007c
:10376000d09d880020332000e09d88001034200088
:10377000f09d880000352000009e88000036200063
:10378000109e8800f0362000209e8800f037200030
:10379000309e880000392000409e8800003a2000ba
:1037a000509e8800103b2000609e8800203c200036
:1037b000709e8800403d2000809e8800503e200082
:1037c000909e8800703f2000a09e8800a0402000ae
:1037d000b09e8800d0412000c09e88000043200099
:1037e000d09e880030442000e09e88007045200074
:1037f000f09e8800b0462000009f8800004820000e
:10380000109f880050492000209f8800a04a200077
:10381000309f8800004c2000409f8800604d2000b1
:10382000509f8800c04e2000609f880030502000cc
:10383000709f8800a0512000809f880020532000a6
:10384000909f8800a0542000a09f88003056200040
:10385000b09f8800c0572000c09f880050592000aa
:10386000d09f8800f05a2000e09f8800a05c2000d4
:10387000f09f8800405e200000a0880000602000cb
:1038800010a08800c061200020a088008063200074
:1038900030a088005065200040a0880020672000ec
:1038a00050a088000069200060a08800f06a200015
:1038b00070a08800e06c200080a08800d06e2000fe
:1038c00090a08800e0702000a0a08800e072200096
:1038d000b0a0880000752000c0a0880020772000dc
:1038e000d0a0880040792000e0a08800807b2000e4
:1038f000f0a08800b07d200000a18800f07f2000ab
:1039000010a1880000000600ffff370006d2bf00ac
:103910000552e300070032000672ec0006d2bf0039
:103920000080fb004162210060c0780023f2b700f4
:103930000100370023f2ef000000060014cea900ba
:10394000462cef00e431ef0011e1a9002132a9007b
:10395000140ea90014cea8001772ef0015f2ef00a4
:103960000000060014cea900462cef00662cef00e4
:10397000e431ef0011e1a900140ea90014cea80053
:103980001772ef00008ea900048ea9000000370016
:1039900014cea90000052000608f8800628f80008f
:1039a000020141004032210060007900306388004c
:1039b00040c0b3001cf2b70040c1b3001df2b70015
:1039c0001b000700e0c1b30018f2b70018d2bf0017
:1039d0000080fb000020ec004400dd00f08e880039
:1039e00040c1b30019f2b70040c6b3001af2b700e5
:1039f00080c0b3001bf2b70010c0b300ee51b50099
:103a000005003200c0fd070010c0b300eef1b700a2
:103a100010c0b300eff1b700e431ef00100ea900c1
:103a2000140ea90014cea8002212a900000006005e
:103a30001cd2bf008080fb001dd2bf000080fb00b5
:103a40000200bc000200e00022003600618f80000e
:103a50001cd2bf000080fb00810f50000200360026
:103a60001e72ef00030037001cd2bf00ec51b500fe
:103a70001ef2b700618f80001cd2bf000080fb00e7
:103a80000100400080007800f0072000808f500087
:103a900003003600f0c7b3001ff2b7000300370081
:103aa000608f80001c52b4001ff2b7001821ef0095
:103ab0000388a9001dd2bf000080fb000000400069
:103ac0004122210060807800e00888002388a80057
:103ad00005003700628f8000020141004032210062
:103ae0006000790030638800000006001672ef0065
:103af000f0c7b3001652e30016003e00020020009b
:103b000003f8230016d2bf00ccf30700aef2070083
:103b1000020020000330240009f30700808f880092
:103b2000918f8800808f8000918f80004df2070078
:103b30000001be0016d2bf000080fb00c200dd0005
:103b400040422100008040000288be001672ec0056
:083b5000e7ff39000000060048
:020000040000fa
:103b5800ce1100000a00000080000000d81100000b
:103b68001800000080000000f011000014000000a0
:103b78008000000004120000200000008000000007
:103b8800241200000002000080000000241400003d
:103b98000002000080000000241600000001000060
:083ba800800000000000000095
:00000001FF
